:0200000480007A
:100000006F000005732F2034930F80006308FF03F7
:10001000930F90006304FF03930FB0006300FF038E
:10002000130F000063040F0067000F00732F2034CC
:1000300063540F006F00400093E19153171F0000BD
:1000400023223FFC171F000023200FFC6FF01FFF2F
:100050009300000013010000930100001302000050
:100060009302000013030000930300001304000038
:100070009304000013050000930500001306000020
:100080009306000013070000930700001308000008
:10009000930800001309000093090000130A0000F0
:1000A000930A0000130B0000930B0000130C0000D8
:1000B000930C0000130D0000930D0000130E0000C0
:1000C000930E0000130F0000930F0000732540F102
:1000D0006310050097020000938202017390523072
:1000E000735044749702000093820201739052305F
:1000F00073500018970200009382420273905230AE
:100100009B021000939252039382F2FF7390023B82
:100110009302F0017390023A73504030970200004E
:1001200093824201739052307350203073503030BC
:100130009301000097020000938202ED7390523009
:10014000130510001315F501635C05000F00F00F97
:10015000930110009308D005130500007300000000
:1001600093020000638A020073905210B7B200003D
:100170009B829210739022307350003097020000DF
:100180009382420173901234732540F17300203042
:1001900093012000972000009380C0E61301A0FA8D
:1001A0009707000093874701238020000387000002
:1001B0006F008000130701009303A0FA63147744D3
:1001C00093013000972000009380C0E313010000EA
:1001D0009707000093874701A38020000387100042
:1001E0006F0080001307010093030000631C774039
:1001F00093014000972000009380C0E037F1FFFF9B
:100200001B0101FA97070000938747012381200013
:10021000039720006F00800013070100B7F3FFFF72
:100220009B8303FA6310773E9301500097200000F0
:10023000938040DD1301A0009707000093874701DA
:10024000A3812000038730006F00800013070100A6
:100250009303A0006318773A930160009720000091
:100260009380B0DA1301A0FA970700009387470143
:10027000A38E20FE0387D0FF6F00800013070100CC
:100280009303A0FA63107738930170009720000061
:100290009380B0D7130100009707000093874701B0
:1002A000238F20FE0387E0FF6F008000130701000B
:1002B00093030000631877349301800097200000B7
:1002C0009380B0D4130100FA970700009387470189
:1002D000A38F20FE0387F0FF6F008000130701004B
:1002E000930300FA63107732930190009720000087
:1002F0009380B0D11301A0009707000093874701B6
:1003000023802000038700006F0080001307010096
:100310009303A0006318772E9301A000972000009C
:100320009380C0CE375134121B018167138200FEC7
:100330002300220283820000930380076394722CBF
:100340009301B00097200000938040CC373100002B
:100350001B0181099380A0FFA383200017220000C6
:100360001302D2CA83020200930380F9639C7228AD
:100370009301C000130200009300D0FD172100007C
:10038000130141C823001100030701009303D0FDAE
:10039000631A77261302120093022000E31E52FC18
:1003A0009301D000130200009300D0FC172100003D
:1003B000130141C513000000A30011000307110041
:1003C0009303D0FC631077241302120093022000E1
:1003D000E31C52FC9301E000130200009300C0FCF8
:1003E00017210000130101C21300000013000000D8
:1003F00023011100030721009303C0FC631477203D
:100400001302120093022000E31A52FC9301F00041
:10041000130200009300C0FB13000000172100002E
:10042000130141BEA3011100030731009303C0FB78
:10043000631A771C1302120093022000E31C52FC83
:1004400093010001130200009300B0FB13000000B1
:1004500017210000130101BB13000000230211004B
:10046000030741009303B0FB631E771813021200C9
:1004700093022000E31A52FC9301100113020000C2
:100480009300B0FA130000001300000017210000D1
:10049000130141B7A3021100030751009303B0FAFF
:1004A000631277161302120093022000E31A52FC23
:1004B000930120011302000017210000130181B4F1
:1004C000930030032300110003070100930330035E
:1004D000631A77121302120093022000E31E52FCEB
:1004E000930130011302000017210000130181B1B4
:1004F0009300300213000000A30011000307110055
:10050000930330026310771013021200930220004D
:10051000E31C52FC9301400113020000172100006C
:10052000130141AE930020021300000013000000ED
:100530002301110003072100930320026314770CA9
:100540001302120093022000E31A52FC930150019F
:1005500013020000172100001301C1AA13000000BC
:1005600093002001A3011100030731009303200130
:10057000631A77081302120093022000E31C52FC56
:10058000930160011302000017210000130181A7ED
:10059000130000009300100113000000230211005B
:1005A0000307410093031001631E77041302120036
:1005B00093022000E31A52FC930170011302000021
:1005C00017210000130101A4130000001300000014
:1005D00093001000A30211000307510093031000C1
:1005E000631277021302120093022000E31A52FCF6
:1005F0001305F00E972500009385C5A0A381A500E3
:10060000631030020F00F00F63800100939111001E
:1006100093E111009308D0051385010073000000D9
:100620000F00F00F930110009308D0051305000090
:0C06300073000000731000C00000000008
:1010000000000000000000000000000000000000E0
:1010100000000000000000000000000000000000D0
:1010200000000000000000000000000000000000C0
:1010300000000000000000000000000000000000B0
:081040000000000000000000A8
:10200000EFEFEFEFEFEFEFEFEFEF0000000000007A
:040000058000000077
:00000001FF
